:03000000020410E7
:0C041000787FE4F6D8FD75815202045795
:10069C0050000000000000000000000000000000FE
:0306AC000000004B
:060807008F907F017E00CE
:03080D000207B728
:0D07E300C2A7120807D2A6120809C2A6225A
:0D07F000D2A7120807D2A6120809C2A6223D
:0805F4008F398B3A8A3B893CE8
:1005FC00E4F53DED7006E53924808004E53924C02E
:10060C00FF1207E3AB3AAA3BA93C120382FF60102E
:10061C001207F07401253CF53CE4353BF53B80E4D6
:01062C0022AB
:0A062D008F228D238B248A25892655
:100637007536007537007538278B398A3A893B85B7
:10064700363C85373D85383E7B017A0079001206B6
:0E065700CC7B017A007900AD23AF220205F4BE
:1006FA007F381207E31208097F0C1207E312080970
:10070A007F061207E31208097F011207E31208099C
:0C071A007F801207E37F017E0002080DC3
:100785008F1A531A0F530501ED7004E51A8004E51D
:0A0795001A24404480FF1207E322FB
:0A07FD008B1B120785AF1B0207F0EB
:10079F0046554E3A4F4E0046554E3A4F4646004745
:0807AF00656172733A256400D4
:1006AF00020E0000011100C10AC109010803021264
:0C06BF000000020903E8011000010B001C
:1007B700D3EF9400EE64809480400B7D6EDDFEEFF6
:0607C7001F70ED1E80EA28
:0107CD002209
:10056C0020B71220B742200A3FD20AA209B392093F
:10057C0020B73580FB20B61920B62D200A2AD20AC6
:10058C000508E508D39403400375080120B61980CB
:10059C00FB20B51220B511200A0ED20AE508D3941F
:0905AC00014005150822C20A22D3
:10000E005389F0438901E4F58A758CDCC28DD2A93F
:05001E00D28CD2AF22DC
:03000B0002050FDC
:10050F00C0E0C0D075D000C000758A66758CFC0540
:10051F0010E510D3940A400675100012056C0513F0
:10052F00E51370020512C394E8E5126480948340CA
:10053F0006751200751300D3E513950AE50964805B
:10054F00F8E5126480984004D2B38002C2B3050F5D
:0D055F00E50F7002050ED000D0D0D0E032C4
:10076A0053877F75985053890F438920758BFD7580
:0B077A008DFDC2ABD28ED2AFC2AC220C
:100665008B148A158916AE02AF01EF4E6028C2AC15
:10067500EDD394004020AF051DEF601AAB140516AD
:10068500E516AA157002051514F9120382F59930BD
:0706950099FDC29980E022EB
:10074D008B178A188919AE02AF01EF4E600E120792
:0D075D00CEAD07AB17AA18A9191206652228
:030023000205B51E
:1005B500C0E0C0D030982F85990BE50B249B600FC8
:1005C50024ED6019241E701EA209B3920980170537
:1005D50008E508D39403400E7508018009E508D3A2
:0F05E500940140021508C298C299D0D0D0E032DC
:10049C001206FA12076A7FC87E001207B712000E06
:1004AC00D3E50F94F4E50E6480948140F3E4F50EEB
:1004BC00F50F3009307BFF7A07799FFDFF12062D6F
:1004CC00E50824FE600F14601424027024750901E1
:1004DC00750A2C801C750902750ABC8014750903F9
:1004EC00750AE8800C7BFF7A0779A6E4FDFF1206FB
:1004FC002D7BFF7A0779AE8508277D01E4FF120674
:03050C002D809DA2
:10041C0002049CE493A3F8E493A34003F68001F256
:10042C0008DFF48029E493A3F85407240CC8C333E1
:10043C00C4540F4420C8834004F456800146F6DFB0
:10044C00E4800B010204081020408090069CE47E9E
:10045C00019360BCA3FF543F30E509541FFEE493A5
:10046C00A360010ECF54C025E060A840B8E493A36C
:10047C00FAE493A3F8E493A3C8C582C8CAC583CA97
:10048C00F0A3C8C582C8CAC583CADFE9DEE780BE4F
:0106CB00002E
:10038200BB010689828A83E0225002E722BBFE0279
:09039200E32289828A83E49322AC
:1007CE00E4FFFE120382600C0FEF70010E09E97058
:0507DE00F20A80EF2289
:1006CC00853942853A43853B44EBC53CFBEAC53D45
:1006DC00FAE9C53EF97F097845120382F60809E963
:0E06EC0070010ADFF4AB3CAA3DA93E02008279
:10002600E54E2442F8E6054E22783F300702784234
:10003600E475F0011203DA0203822000EB7F2ED270
:10004600008018EF540F2490D43440D4FF30040BB2
:10005600EF24BFB41A0050032461FFE54F60021578
:100066004F0552E5527002055130070D783FE47591
:10007600F0011203DAEF0203C80207267403D2075F
:100086008003E4C207F54E8B3F8A408941E4F54F71
:10009600F551F552E54F60077F2012006180F57536
:1000A60050FFC201C200C202C203C205C206C20894
:1000B60012002FFF700D3007057F00120072AF523D
:1000C600AE5122B4255FC2D5C20412002FFF24D040
:1000D600B40A00501A75F00A784F30D50508B6FFF5
:1000E6000106C6A426F620D5047002D20380D924C0
:1000F600CFB41A00EF5004C2E5D204020272D20154
:1001060080C6D20080C0D20280BCD2D580BAD205C9
:1001160080B47F201200612002077401B54F0040B1
:10012600F1120026FF12006102009AD208D2068060
:1001360095120026FB120026FA120026F94A4B7089
:100146000679437A037BFF20022EE54F602A7E0064
:100156008E8275830012039B60060EEE655070F06A
:10016600C2D5EBC0E0EAC0E0E9C0E0EE1202B9D0C9
:10017600E0F9D0E0FAD0E0FB120382FF60AAEBC000
:10018600E0EAC0E0E9C0E0120061D0E02401F9D065
:10019600E03400FAD0E0FBE5500460DCD550D980AD
:1001A600877BFF7A0279B5D202809C79108002792A
:1001B60008C206C2088008D2D5790A8004790AC224
:1001C600D5E550047002F550E4FAFDFEFF12002654
:1001D600FC7B08200113120026FD7B1030000A125A
:1001E6000026FE120026FF7B20EC3382D592D550E6
:1001F60013C3E43000069FFFE49EFEE42001039D46
:10020600FDE49CFCE4CBF8C201EC700CCFCECDCC67
:10021600E824F8F870F38017C3EF33FFEE33FEEDF2
:1002260033FDEC33FCEB33FB994002FB0FD8E9EBD3
:10023600300105F8D0E0C448B201C0E00AEC4D4EEA
:100246004F78207B0070C2EAB5500040BCC0E01277
:1002560002BBD0F0D0E0200104C4C0E0C4B201C0AB
:10026600F012004AD0F0D5F0EB02009A1203EA0130
:10027600375301B15801084C01044201B54F01BD85
:0F0286004401BD49011D4301C35501A74601A70E
:100295004501A747036350010C2D01102E01332B97
:1002A500011423013120034C2A00CC480000012B06
:1002B5003F3F3F00790AA2D5200314300509B91044
:1002C500020404B9080104A2D52006025001042045
:1002D50002689202B54F005034C0E07F2030031908
:1002E5007F30A20272067205500F120312C202C2BB
:1002F50006C205C2087F30800F300503E9C0E01251
:100305000061300503D0E0F9D0E0B54FCC300517DA
:100315007F30B9100C1200617F583004077F788058
:1003250003B908031200613002057F2D0200617FC9
:10033500202008F87F2B2006F322920280CF286E1A
:10034500756C6C2900D2011200263001F8C20178C3
:100355004F30D50108F60200CC2D50434958120004
:10036500262403B405004001E490035E9312005275
:0D037500743A120052D203754F040201B118
:10039B00BB010CE58229F582E5833AF583E0225017
:1003AB0006E92582F8E622BBFE06E92582F8E22261
:0D03BB00E58229F582E5833AF583E493227B
:1003C800BB010689828A83F0225002F722BBFE0114
:0203D800F3220E
:1003DA00FAE6FB0808E6F925F0F618E6CA3AF62224
:1003EA00D083D082F8E4937012740193700DA3A3A2
:1003FA0093F8740193F5828883E4737402936860B6
:06040A00EFA3A3A380DFB5
:10072600EFB40A07740D120731740A309811A899AC
:10073600B8130CC2983098FDA899C298B811F63033
:0707460099FDC299F599220B
:00000001FF
